:1000000009C0189518950DC118951895189518954B
:10001000189518958FE98DBFCCE8E1E84E2EDD27C5
:100020005D2EA89584B7082E877F84BF88E1992725
:1000300081BD91BDEEE3F0E0A0E6B0E088278D93AE
:100040003197E9F7662487EE87BB8CEF88BB84E0A5
:1000500083BF80E08FBD89B7826089BF7894A6E3B3
:100060008C9183FBA0E68C9187F98C93A6E38C910D
:1000700084FBA0E68C9186F98C93A2E619D10091BD
:100080006100003009F017C0A0E68C9187FB81E089
:100090000EF080E08F93A0E68C9186FB81E00EF05D
:1000A00080E09F918923882309F404C0A1E68C9104
:1000B0008F5F8C9369C0013009F02BC0A0E68C9152
:1000C00087FB81E00EF080E08F93A0E68C9186FBA9
:1000D00081E00EF480E09F918923882309F403C016
:1000E00082E080936100A0E68C9187FB81E00EF4B2
:1000F00080E08F93A0E68C9186FB81E00EF080E09B
:100100009F918923882309F403C083E080936100D1
:100110003BC0023009F01BC0A0E68C9187FB81E058
:100120000EF480E08F93A0E68C9186FB81E00EF0C8
:1001300080E09F918923882309F408C081E090E042
:10014000A2E68D939C9380E0809361001DC00330F4
:1001500009F01AC0A0E68C9187FB81E00EF080E0E8
:100160008F93A0E68C9186FB81E00EF480E09F9156
:100170008923882309F408C08FEF9FEFA2E68D93AF
:100180009C9380E080936100EF93FF93ECEEF0E0AE
:1001900086D0FF91EF91A2E60D911C91003050E0C6
:1001A000150709F40DC0A2E60D911C91013050E035
:1001B000150709F003C0C098C19A02C0C198C09A3F
:1001C000A0E68C9185FB0EF029C0809160008F7DA8
:1001D00080936000A8E30C9100FB81E00EF080E0CA
:1001E0008F93A8E30C9101FB81E00EF080E09F91DA
:1001F000892B882309F40FC0A5E68C918F5F8C931F
:10020000009165000F3009F005C080E08093650023
:10021000C098C19803C080E08093650020CFF89417
:10022000FFCF0F921F922F923F924F925F927F9239
:10023000AF92BF920F931F932F933F934F935F9370
:100240006F937F938F939F93AF93BF93CF93DF93DE
:10025000EF93FF938FB78F9385E082BF809160000B
:100260008062809360008F918FBFFF91EF91DF914B
:10027000CF91BF91AF919F918F917F916F915F913E
:100280004F913F912F911F910F91BF90AF907F9011
:100290005F904F903F902F901F900F90189531973F
:1002A000F1F70895689462F80895E89462F8089563
:1002B00082E001C084E099279D938A95E9F708952B
:00000001FF
